:1000000085018601831681130030860085008515E1
:1000100006168616831280308C0030200C081D20B6
:10002000861E8C0A061E8C030F300C0203198C0AE4
:10003000C8300C0203198C030D288D008D09262071
:100040008D0B1F2805152B20051108000A308E0086
:100050008E0B282808001E308E008E0B2D280800DD
:10006000851D3528851932280800851D352808008A
:10400000FF3FFF3FFF3FFF3FFF3FFF3FFF3FFA3FC5
:00000001FF
